:020000040000FA
:100000008301242883120D08100203180C280319F9
:100010000C280130900000349001003483120D0848
:100020001002031C1828031918280130900000340E
:100030009001003483120D081002031D22280130A4
:100040009000003490010034BE309F00FA309900D7
:1000500078309A009B011F089800A2010730831690
:100060008500703086008312861006100030061E50
:100070003A2801308312A0000030861E402801304B
:100080008312A1000030061F4628013083129E0013
:100090001E0892000030900012088D001A20831272
:1000A0001008101C562801309C0059288312033078
:1000B0009C008312210892000030900012088D00ED
:1000C0001A2083121008101C6828190897006B2842
:1000D00083121A08970083128312200892000030BE
:1000E000900012088D001A2083121008101C852819
:1000F0000030051C7C280130831294000030851CE0
:100100008228013083129500922883120030051C4A
:100110008A280130831295000030851C9028013018
:100120008312940083120030051D9728013083123A
:1001300096000D308C004A308D008D0B9D288C0B65
:100140009B280000000000000000000000000000EC
:1001500000000000200892000030900012088D007E
:100160001A208312100892001408930001309000A6
:1001700013088D001A208312100812089005101C15
:10018000C7280030051CC528013083129400831253
:10019000200892000030900012088D001A2083126F
:1001A00010089200150893000130900013088D008C
:1001B0001A208312100812089005101CE528003040
:1001C000851CE328013083129500831220089200D9
:1001D0000130900012088D001A208312100892003E
:1001E000150893000130900013088D001A20831227
:1001F000100812089005101C03290030051C012965
:100200000130831295008312200892000130900083
:1002100012088D001A20831210089200140893000F
:100220000130900013088D001A2083121008120864
:100230009005101C21290030851C1F2901308312D4
:100240009400831214089200190893001808900073
:1002500013088D000E20831201309006100812083A
:100260009005101C3829180892001C0812079800E5
:100270008312150892001A089300180890001308BA
:100280008D0002208312013090061008120890059C
:10029000101C4F29180892001C08120298008312A3
:1002A000160892001B0893000030900013088D0080
:1002B0001A208312100812089005101C732914309C
:1002C0009B00210892000030900012088D001A2037
:1002D00083121008101C6F291A08970072298312C4
:1002E00019089700831283121B08920000309000B7
:1002F00012088D00022083121008101C81299B0314
:1003000094298312210892000030900012088D0079
:100310001A2083121008101C90291908970093299D
:1003200083121A08970083128312061401309D006D
:10033000831218081D0203199F299D0A9829831208
:100340000610861401309D00831217081D02031940
:10035000AB299D0AA429831286101C308C00AF3073
:100360008D008D0BB1298C0BAF29220892005A30D9
:10037000900012088D001A2083121008101CC22948
:10038000A201C4298312A20A8312220892005530C6
:10039000900012088D00022083121008920022089B
:1003A00093005A30900013088D000E20831210081D
:1003B00012089005101CDE298611E029831286158B
:0403C00083126C2810
:00000001FF
